:1000000006C2000021C200001FC200001DC2000085
:100010000C94B90E19C2000017C200000C94A80E6F
:1000200013C2000011C200000FC200000DC2000088
:100030000BC2000009C2000007C2000005C2000098
:1000400003C2000001C20000FFC10000FDC10000AA
:100050000C943B0EF9C10000F7C10000F5C100008F
:10006000F3C10000F1C10000EFC10000EDC10000CC
:10007000EBC10000E9C10000E7C1000032303232BC
:1000800030373233303633310040004000400040DA
:100090000040004000400040004000400040004060
:1000A00000400040004000000CA8074409C405318E
:1000B00008240680072206F106F4056E06AE050642
:1000C000055905D2045B04F303960345037E033709
:1000D00003F702BE028A025B0230020A02E701C78E
:1000E00001A9018E0176015F014A01360124011345
:1000F00001030118010901FB000A01FD00F000FCE9
:1001000000F000FF00FF00FF00FF00FF00FF00FF06
:1001100000FF00FF00FF00FF00FF00FF00FF00FFE7
:1001200000FF00FF00FF00FF00FF00FF00FF00FFD7
:1001300000FF00FF00FF00FF00FF00FF00FF00FFC7
:1001400000FF00FF00FF00FF00FF00FF00FF00FFB7
:1001500000FF00FF00FF00FF00FF00FF00FF00FFA7
:1001600000FF00FF00FF00FF00FF00FF00FF00FF97
:1001700000FF00FF00FF00FF00FF00FF00FF00FF87
:1001800000FF00FF00FF00FF00FF00FF00FF00FF77
:1001900000FF00FF00FF00FF00FF00FF00FF00FF67
:1001A00000FF00FF00FF00FF00FF00FF00FF00FF57
:1001B00000FF00FF00000000000000000000000041
:1001C000000000000000000000000000000000002F
:1001D000000000010001000200020003000300040F
:1001E00000040005000500060006000600070007E1
:1001F00000070007000700070008000800080008C3
:1002000000080008000800080008000800080008AE
:10021000000800080008000800080008000800099D
:1002200000090009000A000A000A000B000B000C7C
:10023000000D000D000E000F000F00100011001245
:100240000012001300140015001600170018001902
:10025000001A001B001C001D001E001F00210022B0
:1002600000230025002600270029002A002C002E4C
:10027000002F00310033003500370039003B003DCE
:10028000003F0041004300460048004A004D004F37
:10029000005200550058005A005D0060006300677E
:1002A000006A006D007100740078007B007F00839D
:1002B0000087008B008F00930097009C00A000A592
:1002C00000AA00AF00B400B900BE00C300C900CE50
:1002D00000D400DA00DF00E600EC00F200F800FFD6
:1002E00000010002000400060009000C000F0013CA
:1002F0000017001C002200290030003700400000D9
:100300000CA8074409C4053108240680072206F119
:1003100006F4056E06AE0506055905D2045B04F326
:1003200003960345037E033703F702BE028A025B8E
:100330000230020A02E701C701A9018E0176015FBE
:10034000014A01360124011301030118010901FBCF
:10035000000A01FD00F000FC00F000FF00FF00FFBC
:1003600000FF00FF00FF00FF00FF00FF00FF00FF95
:1003700000FF00FF00FF00FF00FF00FF00FF00FF85
:1003800000FF00FF00FF00FF00FF00FF00FF00FF75
:1003900000FF00FF00FF00FF00FF00FF00FF00FF65
:1003A00000FF00FF00FF00FF00FF00FF00FF00FF55
:1003B00000FF00FF00FF00FF00FF00FF00FF00FF45
:1003C00000FF00FF00FF00FF00FF00FF00FF00FF35
:1003D00000FF00FF00FF00FF00FF00FF00FF00FF25
:1003E00000FF00FF00FF00FF00FF00FF00FF00FF15
:1003F00000FF00FF00FF00FF00FF00FF00FF00FF05
:1004000000FF00FF00FF00FF00FF00FF00001124BD
:100410001FBECFEFCDBFDFE3DEBF18E3A0E0B8E340
:10042000ECE1F4E202C005900D92A232B107D9F7D7
:1004300028E3A2E2B8E301C01D92A73CB207E1F7AE
:100440000E94C90E0C940912DBCDF89498ED94BF6C
:10045000809361008091630080FDFCCF78940895C3
:10046000E4E9F8E320E030E09081992339F02F5F50
:100470003F4F339620313105B9F70BC0F901EE0F2C
:10048000FF1F2E0F3F1FF901EC56F74C808361834D
:10049000728308950F931F93CF93DF93D091943875
:1004A000DD2351F10091953810919638C091713843
:1004B000C150C7FD0DC0EC2FEE0FFF0BEE58F74CEF
:1004C0000190F081E02DB8018D2F09958111F0CFB9
:1004D000E4E9F8E383818083848195818183928339
:1004E000339688E3E13CF807A9F71092C1381092DF
:1004F000C2381092C338D2CFDF91CF911F910F91A4
:100500000895BC018091C638ABCF1092C6381092C6
:10051000C4381092C53881E080934C3808950F9309
:100520001F93CF93C82F02E919E0CC2349F085E04F
:100530008CDFC8010197F1F781E087DFC150F5CF6B
:10054000CF911F910F910895E0E0F6E082858160E0
:100550008287808581608087089586B183FB8827A4
:1005600080F991E0892780936A380895E0910638F0
:10057000F09107383196FB70F460E0930638F09301
:100580000738809166388B5A80936638E491809161
:1005900066388E0F0895809368388093673881118C
:1005A00012C010923C0A10923D0A1092380A109222
:1005B000390A1092200A1092210A909104049D7F1A
:1005C000909304042DC090910404926090930404CD
:1005D0002FEF280F30E0220F331FF901EF51FD4FAD
:1005E0004591549140933C0A50933D0AF901EB54D4
:1005F000FE4F459154914093380A5093390AF901BE
:10060000E757FF4F259134912093360A3093370AEC
:1006100090912B38911104C01092200A1092210A57
:1006200080932B38809168388F3010F485E001C0BA
:1006300081E00BCFCF93DF93CDB7DEB72697CDBF49
:10064000DEBF9091193820918238309183382B5138
:100650003B4009F492E0843019F460934A381FC09B
:100660006623E9F0823019F427E9261B622F26E081
:10067000E6E1F4EADE01119601900D922A95E1F788
:100680009E012F5F3F4F280F311D280F311DF901AB
:1006900032970190F081E02DE90FF11D60832696DD
:1006A000CDBFDEBFDF91CF910895BF92CF92DF9291
:1006B000EF92FF920F931F93CF93DF93EC01409142
:1006C0001938E0911A38EE2311F082E001C0842F2E
:1006D00090E0DC01AD5EB74C2C9120931738DC0123
:1006E000A05FB74C8C9180931638F0E0E35FF74C35
:1006F0003181622F70E0442349F0313039F49B019D
:10070000280F311DC9019595879538C0C617D707A1
:10071000A4F1682F70E06C177D0784F1411102C0CD
:100720008C2F2CC0821B032F10E001501109E82EE2
:10073000F12CC701B8010E94C21160934838669538
:10074000E62FF0E0822FC12CD12CB12CB316B1F0E2
:10075000C601B8010E94AE11822F860FCE0CDF1C9D
:10076000AE01481B510957FF03C0519541955109EE
:10077000E417F5071CF4B394E9CF822FDF91CF91F2
:100780001F910F91FF90EF90DF90CF90BF90089551
:1007900080934B3800CFCF93C091683889E18C0F9C
:1007A000873908F080E0F7DE82E0B9DE8C2FCF9148
:1007B000F2CECF93C091683880E0EDDE83E0AFDE0B
:1007C0008C2FCF91E8CE81E00895611160931F389E
:1007D0000895662389F0813061F480918538909185
:1007E0008438891B681B6093843882E080932038AA
:1007F00003C0635E60931E3880911E38873418F002
:1008000086E480931E3808956093433808950F93CB
:100810001F93CF93DF938091193880934D38809147
:10082000133880934E388091103880934F388091E0
:100830000D388093503880911438809351388091CE
:1008400011388093523880910E38809353388091BC
:1008500015388093543880911238809355388091A0
:100860000F388093563880911A388093573880918A
:100870004A3880935838809149388093593880910C
:10088000183880935A3880911C3880935B38809157
:100890001B3880935C3880910B3880935D38809151
:1008A000093880935E3880910A3880935F38809150
:1008B00008388093603880910C388093613880913B
:1008C0001E38809362388091843880936338809199
:1008D0001F3880936438809143388093653882E074
:1008E0001EDEF8940DE418E3C1E4D0E0F801619154
:1008F0008F01CE010E94EC112196CA35D105B1F7C6
:1009000065EA80E490E00E94EC117894DF91CF9149
:100910001F910F9108951092933890911006809135
:100920006638890F8093663880918838882309F467
:100930000BC11092883880919138811140C080910C
:100940002038882349F080918D3890918E3880939B
:10095000893890938A3804C08091893890918A3878
:100960004096807E9695879567EE72E00E94AE1164
:1009700080911F38680F99EF960F90938738809178
:100980003F38882311F081500AC06D51673010F054
:10099000973038F460E070E084E062DD85E08093B9
:1009A0003F38809169388111C6C08EE18093060678
:1009B00085E48093020681E080939138B9C081304C
:1009C00009F0B9C080912038811143C080918B38E3
:1009D00090918C3840969C0145E0369527954A9534
:1009E000E1F7A0918438A901569547950A2E000C8D
:1009F000BB0BCD0183519140840F951F80938538A7
:100A00009093863880912E38E82FF0E0EE0FFF1F8C
:100A1000E15DF74C40815181B901641B750B208366
:100A200031838F5F877080932E38CB01880F991F99
:100A3000880F991F40911E3850E04D5E5E4F4A1B53
:100A40005B0B440F551F841B950B820F931F23E0F4
:100A50001CC080918F389091903880938B38909300
:100A60008C38409635E0969587953A95E1F7EFE218
:100A7000F8E38193919328E3EF33F207D1F7A6CF00
:100A8000009709F00196215029F018161906C4F7AD
:100A90000197F9CF18161906E4F477FD39C02091B3
:100AA0002D3812160CF1880F991FBC016350710983
:100AB00077FF02C06F5F7F4F759567951616170613
:100AC00014F061E070E088E1861B80932D3885E0AA
:100AD00026C08C3F2FEF9207DCF477FF19C02091DE
:100AE0002D3827FF05C02450281B20932D3818C00F
:100AF00024EE281B20932D38209187382F3180F049
:100B00006CEF7FEF681B790B7595679586E007C0E2
:100B1000809187388E3120F060E070E087E0A0DCC3
:100B200089E08093060685E480930206109291384E
:100B30001092923809DD80912038882329F0809125
:100B400020388150809320380895813019F4109214
:100B50001C380895823019F460931B38089583304F
:100B600019F4609349380895843011F4609318386B
:100B70000895CF93C0911A38C1114AC0883039F412
:100B800010924738109244381092453842C0813B49
:100B900059F48091473881508330D0F583E08093B9
:100BA00047388093463834C0853BB1F4CB016EE3BF
:100BB00070E00E94AE11892B61F5809147388A3F21
:100BC00040F58B5F809347388093463810924438C5
:100BD00010924538E0DD1DC08130D1F48091443859
:100BE00090914538019688382EE0920728F480933A
:100BF0004438909345380DC01092443810924538CF
:100C000080914738882329F081508093473801C06C
:100C1000C1E08C2FCF910895FF920F931F93CF9334
:100C2000DF938C01EB01F42E809182389091833810
:100C3000892B31F0E0918238F091833889E0099571
:100C40000093823810938338012B39F0E091823879
:100C5000F0918338BE018F2D099581E080934C3847
:100C6000DF91CF911F910F91FF900895CF93DF9364
:100C7000E0917138EE2359F0E150E0937138F0E0E3
:100C8000EE0FFF1FEE58F74CC081D18102C0C0E0CB
:100C9000D0E0E0917138EE2341F0F0E0EE0FFF1F5D
:100CA000E059F74C8081918102C080E090E04AE0F9
:100CB00060E070E0B1DFCE01DF91CF910895883020
:100CC00029F4109240381092263815C08130F9F47A
:100CD00090912638911107C06032710568F18093B8
:100CE000263813DC29C0913081F46B3B710528F064
:100CF00082E08093263880E01EC061157105E1F026
:100D00006270862F880F8E5E16C0B0DF15C08138E6
:100D100011F0813E89F491E090932638813E21F4D0
:100D200080914038865F03C0809140388F5F809308
:100D30004038EBDB8BE42FDC80E008959C01909140
:100D40007138983088F4E92FF0E0EE0FFF1FEE586D
:100D5000F74C208331839F5F9093713848E0C9013D
:100D60005BDF8091713808958FEF08950F931F9383
:100D7000CF93DF93EC018B0179DFB801CE01DF91D6
:100D8000CF911F910F91DACF813C29F460E070E0A0
:100D900082EC97E006C0823C39F460E070E085E2C6
:100DA00097E0E4DF80E0089581E00895843011F554
:100DB00080918238909183382CE08F36920729F405
:100DC00069E170E082E998E013C08259984061F4CB
:100DD00090916838923040F0892F86959695969537
:100DE000890FD6DC80E0089560E070E082EC97E047
:100DF000BDDFF8CF81E00895813C29F460E070E028
:100E000082EC97E006C0823C31F460E070E084EC54
:100E100096E0ACDF16C0813B49F4CB016EE370E095
:100E20000E94AE11892B69F4B6DC0BC0813E59F4E7
:100E3000CB016EE370E00E94AE116F5F60930C38DF
:100E4000E6DC80E0089581E00895CF93C0911A38E0
:100E5000C11117C0813C29F460E070E082EC97E09A
:100E600006C0823C31F460E070E085E497E07EDF0C
:100E700009C0873B31F460E070E083E29BE05EDF15
:100E800001C0C1E08C2FCF910895813C29F460E02E
:100E900070E082EC97E006C0823C31F460E070E0E4
:100EA0008CEF96E063DF07C0873B39F460E070E0C9
:100EB00087E29BE043DF80E0089581E00895CF93CF
:100EC000DF93D82F80798039A9F42091133890913D
:100ED00014388D2F8F70823041F480911C3881112D
:100EE0000CC0822F291748F403C0822F921728F4D0
:100EF000892F03C0803819F480E04DDB08C0D13061
:100F000031F469317105B8F1D093693834C0D33CFC
:100F100031F441DC60E070E082EC97E01EC0D43C2C
:100F200071F4C0911C38CC2319F06C2F70E013C001
:100F300060911D3870E082E998E018DF1FC0D43B53
:100F400031F437DC1092C63861E070E004C0D53C63
:100F500031F466E970E082E998E008DF0CC0C091E6
:100F60001A38C1110AC0DA3B41F460E070E08BE24C
:100F70009BE0E4DE03C0C0E001C0C1E08C2FDF9144
:100F8000CF9108950F931F93CF938B01883059F41D
:100F900080E001DB10924738012B19F481E0809347
:100FA0006938C0E0BAC0813021F469317105C8F3F5
:100FB000F6CF833009F580911C38882371F0909129
:100FC0001B3842EC51E0949F9001959F300D112405
:100FD0006217730710F080931D388091433888237F
:100FE00001F342EC51E0849F9001859F300D112464
:100FF00020173107B0F64CC0813B91F481E090E0BE
:1010000054DBC9DA809149388111CBCF80911938EE
:10101000811103C00831110520F261E070E028C0A1
:10102000813ED9F3813821F480911D3890E013C0BE
:10103000813C21F46091683870E01AC0823B79F4F9
:101040008091183890911A38911180914A38811105
:1010500004C086E990E029DB05C086E903C0823E32
:1010600019F480E098DA9DCF823C29F466E970E0BB
:1010700082E998E008C08339A1F3833C31F460E051
:1010800070E085E297E072DE8CCF843C31F483DB44
:1010900060E070E08FE597E0F6CF8D3B49F4F8947F
:1010A00088ED84BF81E0809300017894A895FFCFFC
:1010B0008F3C29F460E070E083EE93E0E4CFC091D0
:1010C0001A388A3B79F4672B69F4CC2329F063DB67
:1010D00010921A389CDB65CF60E070E08BE19BE0FA
:1010E0002DDE1BC0C11118C08A3C31F454DB81E0F5
:1010F00080931A388CDB11C0833B29F460E070E0E8
:101100008FE69CE007C0853C39F445DB60E070E089
:1011100087EF9DE02BDE01C0C1E08C2FCF911F91A6
:101120000F9108959F92AF92BF92CF92DF92EF926C
:10113000FF920F931F93CF93DF93182FEB01D09063
:101140001738F0901638A0901938AA2019F0B090EE
:10115000483802C0BB24B394C090183800911A38A4
:101160000111C0904A38CC2051F041E0C41621F062
:1011700080911D388F1518F0A6E9EA2E01C0EF2CDA
:1011800090904738BE01812FF4DC2091473822230C
:1011900039F091100CC08091683880932A3807C0CC
:1011A000992029F060E070E082EC97E039C0812F4F
:1011B0008D7F8830D9F4109242381A3019F4C091DA
:1011C0001D38D0E08D2D90E08C179D0738F48F2DC1
:1011D00090E0C817D90710F4C0931D38CE0165DA26
:1011E000D7DA81E08093053800E0D0C1113CD1F21C
:1011F000123C71F4809168388E1510F48E2D02C067
:1012000080911D38C5DA8091683880932A38ECCFF8
:10121000143C41F480E0BFD960E070E08FE597E0D6
:10122000A5DDE2CF8FE4810F823008F04FC0AA2005
:1012300041F0CE0168E170E00E94AE11892B31F0DF
:10124000D3CF60910D3870E0CE01F6CF8091683831
:10125000209761F4123B11F48FEF05C08F15E0F772
:10126000D81648F181E08093053825C020910D38CB
:1012700030E066E371E0269FA001279F500D369F66
:10128000500D11244C175D0710F48F1528F76CE6EC
:1012900072E0269FA001279F500D369F500D11240C
:1012A0004C175D0740F4D81630F075DA60E070E056
:1012B0008FE597E05BDD30910538209168384B2D44
:1012C0003403C0011124820F911D26C18FE1810FCB
:1012D000823020F480910538819584CF113009F057
:1012E000CFC0A99711F4109305382223B1F0409193
:1012F0002A3830E021503109429FC001439F900DB0
:1013000011246091463870E00E94C211611101C041
:1013100061E06093673860934B38C09167382091E3
:1013200068388C2F90E0821B910960912838709169
:1013300029386F5F7F4F6093283870932938009762
:1013400009F452CF97FF05C02A3630F040E450E050
:1013500005C040E052E002C040E051E0569547959C
:1013600097FD0196959587950097C1F74617570702
:1013700008F03ACFC21710F48FEF03C02C1718F4FF
:1013800081E0820F01C08C2F9FEF980F492F50E012
:10139000440F551FBA016F517D4FFB01A591B491C8
:1013A000921770F420913C0A30913D0A232B41F4AE
:1013B000AF3FB10529F4A0933C0AB0933D0A1FC08A
:1013C00020913C0A30913D0A2A173B0738F42091BE
:1013D0003C0A30913D0A2F5F3F4F0DC020913C0ADF
:1013E00030913D0AA217B30750F420913C0A309186
:1013F0003D0A2150310920933C0A30933D0A9A015D
:101400002B543E4FF90145915491E091380AF091E7
:10141000390AE417F50738F44091380A5091390A2F
:101420004F5F5F4F0DC0E091380AF091390A4E17B7
:101430005F0750F44091380A5091390A41505109E0
:101440004093380A5093390AA0913C0AB0913D0A62
:10145000FB0145915491A417B50769F44091380AEE
:101460005091390AF901259134914217530719F423
:1014700092D8C09367381092283810922938B4CE89
:101480001530A9F480916838823408F4ADCE90E02C
:101490008C1B9D0B282F813491052CF087399105E9
:1014A00018F026E901C021E4209367389DCE16305C
:1014B000B1F49091683880914B38981708F094CE29
:1014C000C90FD11D90E08C179D0734F0C134D105B0
:1014D00024F4C1E4D0E001C0EC018C2F0EC0173021
:1014E00079F49091673880916838891710F48F5F8C
:1014F00004C0981708F078CE81508093673874CE76
:10150000133C71F481E0A11080E0809319387FD9F9
:1015100050D98091683890E0C8D880931D3872CE39
:10152000011133C0133B49F4CD2B09F05DCECC2023
:1015300011F086E9E82E8E2D04C0133E21F480912F
:101540001D3826D923C0153C41F480E024D860E042
:1015500070E087EF9DE00ADC19C0173B29F460E0DA
:1015600070E087E19BE00FC01A3C39F48091683845
:1015700080931C384CD90FD909C01A3B31F460E074
:1015800070E08FE19BE0DADB01C001E0802FDF91AA
:10159000CF911F910F91FF90EF90DF90CF90BF9070
:1015A000AF909F900895883069F41092273880E0BA
:1015B0000E94CB0280916A38811137C081E080930C
:1015C000273823C0982F907F903BB9F4209127387B
:1015D000421778F0CB016DE570E0C0D6029739F480
:1015E0002F5F20932738421700F188E303C082E180
:1015F00001C080E00E94CB0218C0903E61F480914F
:101600002738882389F0481778F060E070E08FE58C
:1016100096E094DB0AC08A3041F4609140388091B2
:101620002738F9010995F3D821DB80E008952AE1F4
:1016300033E043E0B8CF2AE133E044E0B4CF25EA19
:1016400035E044E0B0CF25EE33E041E0ACCF29EE09
:1016500033E042E0A8CF24E034E041E0A4CFCF93D0
:10166000DF93C0E0D6E089E08E8385E48A83109220
:101670009138109292380E94A402E0EAF0E0808152
:101680008061808383E08883888581608887DF919B
:10169000CF9108950F931F93CF9310926C38809140
:1016A000C4389091C5389C012F5F3F4F88279078B0
:1016B000822B932B8093C4389093C538C0916A389D
:1016C0000E94AD02C81731F11092693880936A38D0
:1016D0009091C638882359F0892F80699F709F3078
:1016E00009F08F5F8093C63880E090E00DC0892FAD
:1016F0008F7E95FD02C0806801C0806C8093C638E3
:101700008091C4389091C5380E9481021092C438EB
:101710001092C5380091C4381091C538809169384D
:10172000882349F0B80183E00E943002CF911F91D5
:101730000F910C944A02C091C6388C2F807F803B59
:1017400019F460E070E001C0B80181E00E9430024D
:10175000C4FF13C0C5FF02C0C8010CC00831110589
:10176000E0F01092C4381092C538C062C093C638F9
:1017700080E090E00E94810210C0CC2371F0C5FD92
:101780000AC00231110548F0C064C093C63880E039
:1017900090E00E9481020E948502C0912C38C11104
:1017A00005C00E94A40281E080938838CF5FCF718A
:1017B000C0932C38CF911F910F9108958091933849
:1017C0008111A9D880916C38811164CF0895EF926E
:1017D000FF920F931F93CF93DF93EC010AEC18E075
:1017E00082E3E82E82E0F82E2097D9F080914C38E1
:1017F000811119C0809168388F3028F485E00E94EB
:101800002502C70104C081E00E942502C80101979A
:10181000F1F781E00E942502D1DF0E944A02219760
:10182000E3CF81E001C080E0DF91CF911F910F9164
:10183000FF90EF900895CF93C82F882391F089E10E
:101840000E94CB0286EA90E0C2DF80E00E94CB02D9
:101850008AEF90E0BCDFC15091F78AE992E0CF9126
:10186000B6CF89E10E94CB0288E090E0B0DF80E053
:101870000E94CB028AEF90E0AADFEFCFCF93DF93F5
:1018800064E660D5282F892F6AE05CD5EC0122231D
:1018900041F0822FD0DF8C2FCEDF8D2FDF91CF91C3
:1018A000CACFC111F8CFF9CFCF93DF93D82FC3E0C0
:1018B00080911D380E94CB0288EC90E088DFDD2308
:1018C00019F080E991E083DF80E00E94CB0288EC90
:1018D00090E07DDFC15061F7DF91CF910895DF92F5
:1018E000EF92FF920F931F93CF93DF93D82F8B012B
:1018F000C0910B3881E080934238C33009F0E2C0D8
:10190000F09047388D2F35D9FF2051F0809147381E
:10191000811106C060E070E082EC97E027DAD2C067
:10192000D83021F481E080930338CEC0D23C19F442
:1019300010924738D7C0D13BC1F490910238012BA7
:1019400049F4953510F08FEF03C0923018F481E020
:101950008093033880910338890F11F481E03CC1F2
:10196000863508F439C185E537C1D13E31F480911F
:101970000338819580930338ECC0D23B61F481E059
:101980008093033880910238823008F4EAC0815095
:1019900080930238E6C0D13009F0F4C00932110555
:1019A00011F4D0930338D09025388D2D880FD7FCB3
:1019B00080952FE0829FC0011124E09024382E2DC5
:1019C000220FE7FC2095D09101382D9F9001112422
:1019D000232F290FF09023388F2D880FF7FC809547
:1019E000C09100388C9FC0011124822F890F609113
:1019F000023870E0680F711D809147388130B9F46A
:101A0000809144389091453825E0969587952A95A0
:101A1000E1F724E730E0A901481B590B469FC001BC
:101A2000479F900D569F900D1124B90197D4862F92
:101A30000E94CB0200FD06C00E94B6028170D80E43
:101A4000D092253880912238E80EE09224380E9406
:101A5000B60265E277D4F90EF09223380E94B602FE
:101A60008F7331F40E94B6026DE06CD490932238EB
:101A7000DD2339F00E94B6028F7319F4D150D09350
:101A800001380E94B602811108C00E94B60266E1C8
:101A900059D49093013810922438C33038F00E9402
:101AA000B6028F7119F4C150C09300380E94B6027B
:101AB0008F7709F07CC00E94B6026CE043D490930B
:101AC000003875C0D83021F481E08093043886C096
:101AD000D13C31F460E070E082EC97E047D97EC001
:101AE000D23C49F48C2F90E0019665E070E04AD436
:101AF00080930B384CC0D13B51F5C23090F400FDBF
:101B00006DC0EC2FF0E0E75FF74C808190910438D6
:101B1000891B883020F08F3F99F58EEF31C088E027
:101B20002FC0C43009F05AC0909108388091043811
:101B3000890F823010F482E003C0893708F088E70B
:101B400080930838809108380E94CB0247C0D13E6C
:101B500031F48091043881958093043818C0D23BC9
:101B6000A1F481E080930438C23068F500FD36C0EE
:101B7000EC2FF0E0E75FF74C80818F3F79F18F5FCA
:101B800080832CC0D13C09F4A5CFD23E19F40E9429
:101B9000070424C0D53C39F460E070E087EF9DE095
:101BA000E5D880E0D1CFD13011F081E018C0093202
:101BB000110519F481E08093043880916638080F8C
:101BC000009366380BC0C43049F4809108388330E4
:101BD00008F4B8CF8150B4CF8093023880E0DF9111
:101BE000CF911F910F91FF90EF90DF9008950F9389
:101BF0001F93CF93DF93D82F8B01883031F48091DE
:101C00004238813011F488E06ADE8D2F8079803986
:101C100061F481E080934138C0914238C1110CC019
:101C200080911D380E94CB0220C0803839F4109278
:101C3000413880E00E94CB02C0E017C0D130A1F44F
:101C4000C0914138CC2351F0809142388130A1F7C6
:101C5000B801DF91CF911F910F9141CE0733114011
:101C600058F3D093693801C0C1E08C2FDF91CF9138
:101C70001F910F9108951F920F920FB60F9211248A
:101C80002F933F934F935F936F937F938F939F9384
:101C9000AF93BF93EF93FF9381E080930B06809106
:101CA0009238882309F440C0E0919138E130D1F4B2
:101CB0008091211120912011A0911006B091110660
:101CC000A81BB10987FDB39530E06FD3DC01CB01D0
:101CD00080589F4FAF4FBF4F892F9A2FAB2FBB27F5
:101CE000BC0104C0609110067091110686E0660F79
:101CF000771F8A95E1F7F0E0EE0FFF1FDF01A35792
:101D0000B74C6D937C93E757F74C80819181861790
:101D1000970708F401966817790708F401978083FC
:101D2000918381E08093933881E080939238FF9192
:101D3000EF91BF91AF919F918F917F916F915F9143
:101D40004F913F912F910F900FBE0F901F901895BC
:101D50001F920F920FB60F9211248F9381E0809300
:101D6000530180936C388F910F900FBE0F901F908E
:101D700018951F920F920FB60F9211248F933B9AD2
:101D800081E080936B388F910F900FBE0F901F9062
:101D90001895F89480914000877F8093400088EDEB
:101DA000A89584BF90910001907F9093000121E05D
:101DB00030E084BF2093610082E080B981E284B981
:101DC00088E080931004809312048093130480931E
:101DD0001404809315048093160480931704809351
:101DE00031048093320499E090933304809350043B
:101DF00080935104809352048093530484E0809331
:101E0000020287E58093010A8FEF90E08093360A03
:101E10009093370A91E09093000A80913304816097
:101E20008093330490935201809151018111FCCF32
:101E300081E48093500113DC789481E00E948F024A
:101E400060E070E086ED96E00E949E0610924C38AD
:101E50000E94CB030E94AD0281110BC082E00E9460
:101E60008F02F89480E490E0AFD2853AA9F178949B
:101E7000A5C0C0E08C2F0E94CB0283E190E0A7DCDC
:101E80008C2F86950E94CB0283E190E0A0DC0E941B
:101E9000AD028823B9F0CF5FC03461F76091853817
:101EA00080918438681B81E00E94E9030E94070446
:101EB000C6E98C2F0E94CB0284E090E088DCC15000
:101EC000C1F7CCCFCC2351F28C2F0E94CB028DE0F6
:101ED00090E07DDCC150F6CF0DE418E3C1E4D0E022
:101EE000CE0172D2F80181938F012196CA35D105B6
:101EF000B9F7789480914D388093193880914E3895
:101F00008093133880914F388093103880915038E7
:101F100080930D38809151388093143880915238D5
:101F2000809311388091533880930E3880915438C3
:101F300080931538809155388093123880915638A7
:101F400080930F388091573880931A388091583891
:101F500080934A38809159388093493880915A3813
:101F60008093183880915B3880931C3880915C385E
:101F700080931B3880915D3880930B3880915E3858
:101F80008093093880915F3880930A388091603857
:101F9000809308388091613880930C388091623842
:101FA00080931E38809163388093843880916438A0
:101FB00080931F38809165388093433880911C3816
:101FC000811180931D3861E070E082EC97E00E94FF
:101FD0009E06442443945524539447E0242ECC2455
:101FE000C394D12C65E0362E7CEF672E73E0772EFC
:101FF000E8EE8E2EE3E09E2EF2ECAF2EF7E0BF2E41
:102000000E944A0280916F3890917038009751F089
:1020100060916D3870916E380E94B60610926F38DC
:102020001092703880916938882309F45EC080E08E
:102030000E94CB0240925201809151018111FCCF4C
:10204000F9E5F0935001809100068E7F80930006A1
:102050000E94AD028111FCCF0E9485028091330461
:102060008160809333041092933810926C381092F0
:102070006B3880916938882331F180915000897FD5
:102080008460809350008091500081608093500064
:102090008895809150008E7F8093500080916B389E
:1020A00081111092693880919338882331F05092D1
:1020B0002038509288380E948B0480916C38882395
:1020C000C1F2E8DAD6CF22E02093203880913304A1
:1020D000887F80933304C3DA40925201809151018A
:1020E0008111FCCF31E43093500168DB10924C3801
:1020F0008091823890918338E3E0833E9E0779F4A3
:10210000CCE7D0E0FE018491805395DB8CE291E036
:102110005EDB2196F0E0C838DF07A1F7C6C02CE0EF
:102120008F36920779F03DE0873F930709F0B2C000
:1021300080914238813009F0F4C080914138882381
:1021400009F4EFC0C0910B38C23011F120F0C43057
:1021500009F483C055CFEC2FF0E0E75FF74CD08156
:1021600086E90E94CB02C11109C0DA3220F4C30112
:102170000197F1F707C081E090E003C08D2F8695AD
:1021800090E025DB81E00E94CB028D2F90E0C7C05C
:102190000E94B6028F73E82EF12C0E94B602622DC7
:1021A000D1D0E60102C0CC0FDD1F9A95E2F70E9464
:1021B000B602632DC7D0F60102C0EE0FFF1F9A953D
:1021C000E2F7CE0FDF1F0E94B60290E0BE01DAD028
:1021D000C80FD91FC739D10514F0C6E9D0E08C2F3C
:1021E0000E94CB02C701F3DA8E0133E01595079503
:1021F0003A95E1F7011101C001E010E0C701E7DA0B
:10220000C01BD10BD7FF02C0C0E0D0E08C2F0E94D2
:10221000CB020E94B602837039F4C701D8DACE012E
:10222000959587950E94CB02C230D1053CF70E945C
:10223000B6026DE087D0E60102C0CC0FDD1F9A9593
:10224000E2F70E94B60290E0BE0188D0C80FD91F05
:1022500080E00E94CB02CE0162C0C0910838CC0F52
:10226000C73908F0C6E9D4E08C2F0E94CB0285E084
:1022700090E0ADDA809108380E94CB0281E490E0D2
:10228000A6DAD15089F780ED92E0A1DA80E00E94D1
:10229000CB02B6CEF7E085329F0781F48091873874
:1022A000EDDA80911A38882381F0A0926F38B092CD
:1022B000703810926D3810926E38A2CE27E08534B7
:1022C000920731F480918538D9DA88EE93E027C0FF
:1022D00036E08C3F9307C1F480916A38811190CE2B
:1022E00080911D380E94CB0284E690E070DA80E095
:1022F0000E94CB0220910C38289DC001299D900D91
:102300001124845691090BC0845C964051F480E0FE
:10231000CBDA81E0C9DA80E0C7DA80ED97E057DAFE
:102320006FCE80915000897F809350008091500043
:102330008160809350008895809150008E7F8093BB
:1023400050005ECE991B79E004C0991F961708F0E3
:10235000961B881F7A95C9F780950895AA1BBB1B09
:1023600051E107C0AA1FBB1FA617B70710F0A61B95
:10237000B70B881F991F5A95A9F780959095BC01B6
:10238000CD01089597FB072E16F4009406D077FD33
:1023900008D0E4DF07FC05D03EF4909581959F4F6F
:1023A0000895709561957F4F0895A29FB001B39FE6
:1023B000C001A39F700D811D1124911DB29F700D4E
:1023C000811D1124911D089503D0808199270895BE
:1023D000FC01E050FC4E0895262FFADF0080021623
:1023E00011F004D0019701970895262FAF93BF9362
:1023F000E0E0F0E1328131FDFDCFDC01A050BC4EC8
:102400002C932DE924BF23E020830196BF91AF9147
:062410000895F894FFCFCF
:06241600133810380D38E8
:10241C000C161801010100040F29430302010705E2
:10242C0096969601010F96010101010A324B2D0778
:02243C0002009C
:00000001FF
